:100000000C947B030C94B3030C94B3030C94B303D0
:100010000C94B3030C94B3030C94B3030C94B30388
:100020000C94B3030C94B3030C94D61D0C94181DBC
:100030000C9480170C94B3030C94B3030C94B30387
:100040000C94B3030C94B3030C94B3030C94B30358
:100050000C94B3030C9442170C94B3030C94B303A5
:100060000C94B3030C94B3030C94B3030C94B30338
:100070000C94B3030C94B3030C94B3030C94B30328
:100080000C94B3030C94B3030C94B3030C94B30318
:100090000C94B3030C94B3030C94B3030C94B30308
:1000A0000C94B3030C94B3030C94B3038005F405D0
:1000B0008805520556058C0559058F059A05640576
:1000C000EA0568059E056C05A205CC057005A60528
:1000D000D6057605AC05B6055D0593056005960564
:1000E0007B05B105C205E205E4054E058405FD0565
:1000F0001D0623060F05170629062F0635064E0690
:10010000740679067E06830688068D069206970693
:100110009C06A106690769079C079C071B0835090F
:10012000350935093908AD08BE08BE08AF0CB20C58
:10013000EE0C0E0D150D200D230D230D230D3A0E83
:100140003A0E9F0DA20DA70DCD0DF00DF30DF60D7E
:100150001A0E281B4F1B001D4F1B001D9B1BBE1B97
:10016000001DB41CC41C00000000000000000000C2
:10017000000000000000000000000000000000007F
:10018000000000000000000000007E0F00D4FFFF10
:10019000FFC70000007800000000000000002A2BCC
:1001A0002800000000000000000000000000000027
:1001B0000029000000002C1E342021222434262790
:1001C000252E362D3738271E1F20212223242526B1
:1001D0003333362E37381F0405060708090A0B0C7F
:1001E0000D0E0F101112131415161718191A1B1CC7
:1001F0001D2F3130232D350405060708090A0B0C85
:100200000D0E0F101112131415161718191A1B1CA6
:100210001D2F3130354C1E0F0500047F3F1F643207
:1002200014643214783C1E1E140A05222325262845
:10023000292A2C2D2F3032333536383A3B3D3E407B
:1002400042434547494A4C4E5051535557595A5CC1
:100250005E6062646668696B6D6F71737577797BD8
:100260007D7F81838587898A8C8E90929496989AD7
:100270009C9E9FA1A3A5A7A8AAACAEAFB1B3B4B6EC
:10028000B8B9BBBCBEBFC1C2C3C5C6C7C9CACBCC47
:10029000CDCED0D1D2D2D3D4D5D6D7D7D8D9D9DA1A
:1002A000DADBDBDBDCDCDCDCDCDDDDDDDDDCDCDC8F
:1002B000DCDCDBDBDBDADAD9D9D8D7D7D6D5D4D3B7
:1002C000D2D2D1D0CECDCCCBCAC9C7C6C5C3C2C18C
:1002D000BFBEBCBBB9B8B6B4B3B1AFAEACAAA8A7E9
:1002E000A5A3A19F9E9C9A98969492908E8C8A89A1
:1002F000878583817F7D7B79777573716F6D6B697E
:1003000068666462605E5C5A5957555351504E4C52
:100310004A4947454342403E3D3B3A383635333201
:10032000302F2D2C2A2928262523222B0014001AB1
:10033000000800150017001C0018000C0012001324
:10034000002A005F00470004001600070009000AA9
:10035000000B000D000E000F00000028005C00E103
:100360000000001D001B0006001900050011001010
:10037000003600215252005900E000E300E2000084
:10038000002C42000000002C000000E6005000514C
:10039000004F00000061005E0000005B00000000F4
:1003A000003700000060005D005A0062003A003B28
:1003B000003B003D003E003F00400041002F003068
:1003C000002D002E0053001E001F002000210022DF
:1003D00000230024002500260027000000E500017E
:1003E00000010000000100010001000100010033D4
:1003F000003400380001004B000100010001000141
:100400000000000100000000002C00000001004A74
:10041000004E004D00000039000100000001000006
:100420000000000100000047000100010001000180
:1004300000010001000100010001000100010001B4
:1004400000010001000100010001000100010001A4
:100450000001000100010001000100010000000195
:100460000001000100000020782178227833780113
:100470000001000100010001000100010001000174
:1004800000010000000100000000002C000000013D
:100490000001000100010000000100010000000156
:1004A0000000000000010000000100010001000147
:1004B0000005010980A101850319012AB700150172
:1004C00026B700950175108100C0050C0901A10136
:1004D000850419012AA002150126A00295017510B4
:1004E0008100C00660FF0961A1010962150026FFB5
:1004F000009520750881020963150026FF009520EC
:1005000075089102C005010906A101050719E02936
:10051000E71500250195087501810295017508818F
:10052000010507190029FF150026FF00950675082B
:10053000810005081901290515002501950575019A
:100540009102950175039101C009025B000301004E
:10055000A0FA0904000001030101000921110100B2
:10056000012244000705810308000109040100027B
:100570000300000009211101000122220007058269
:100580000320000107050303200001090402000104
:100590000300000009211101000122320007058437
:1005A00003200001120100020000000850414C45E8
:1005B000010001020001120345006C006F006E0093
:1005C00067006100740065000000200341006300C3
:1005D0006800650072006F006E002000500072001D
:1005E0006F006A00650063007400000004030904E2
:1005F000FFAA7F5540000101010101010101010233
:1006000002020202020202020303030303030303C2
:10061000040404040404040505050505060606068D
:1006200006070707070708080808090909090A0A49
:100630000A0B0B0B0C0C0C0D0D0D0E0E0E0F0F0FED
:100640001010111111121213131414151516161778
:1006500017181819191A1A1B1B1C1D1D1E1E1F20E6
:1006600020212222232424252626272829292A2B33
:100670002C2D2D2E2F303132323334353637383958
:100680003A3B3C3D3E3F4041424344454647484952
:100690004A4C4D4E4F50515354555658595A5B5D24
:1006A0005E5F616264656668696B6C6D6F707273C2
:1006B0007577787A7B7D7E8082838587888A8C8E29
:1006C0008F91939596989A9C9EA0A2A3A5A7A9AB5B
:1006D000ADAFB1B3B5B7BABCBEC0C2C4C6C9CBCD4D
:1006E000CFD1D4D6D8DBDDDFE2E4E7E9EBEEF0F3FF
:1006F000F5F8FAFDFF0011241FBECFEFDAE0DEBFF0
:10070000CDBF04B603FE18C08091FC029091FD029B
:10071000A091FE02B091FF028730904BA740B04BF2
:1007200059F41092FC021092FD021092FE021092F7
:10073000FF02E0E0F8E3099511E0A0E0B1E0E2EFAC
:10074000FEE402C005900D92A63AB107D9F722E067
:10075000A6EAB1E001C01D92AC3FB207E1F70E94EA
:1007600090090C9477270C940000A8E0B0E0EBEB24
:10077000F3E00C94EF26FC018481882309F4CCC5B6
:100780007F0121E0408151816281738195810E94C6
:1007900034248C01F7019581992309F438C198011B
:1007A00037572038310508F054C1003108F03FC1F7
:1007B0008FEF93E00E94E425811139C13EEAA32E18
:1007C000BB24B394002379F0A114F4E0BF0609F42C
:1007D0002EC1C5010E94E425811101C001502FEFF7
:1007E000A21AB20AEFCFCE0101962C0188E0F201E5
:1007F00011928A95E9F72AE0322E85010F5F1F4F8B
:10080000C5010E94E42589831A82882309F40FC157
:10081000813009F041C06501F2E0CF0ED11CC80162
:100820000E94E4258A83882309F401C19FEF980F71
:10083000933060F423E0A20EB11CC6010E94E425AF
:100840008B83882309F4F3C01C8229C0843031F5DE
:100850004E0133E0830E911C02E010E056018FEF51
:10086000A81AB80AC6010E94E425F40181934F0139
:10087000882309F4DCC08C3741F4E2E0F0E0EC0FAF
:10088000FD1FE00FF11F10820AC00F5F1F4F6501AF
:100890000730110519F7CBC0580101C0560182017C
:1008A000F8012081222309F4A8CF213009F053C098
:1008B0008181813081F46801F2E0CF0ED11CF80112
:1008C0008281893319F460E570E002C060E070E075
:1008D0000E94052415C0823049F46801F2E0CF0E71
:1008E000D11CF80182810E9449230AC0833051F44F
:1008F0006801F2E0CF0ED11CF80182810E94F8223B
:10090000860182C0843019F00F5F1F4F7DC0F8014F
:1009100022810E5F1F4F80E090E030E020533109CC
:100920002A30310568F4389EA001399E500D1124FB
:10093000C901840F951F0F5F1F4FF8012081EDCF74
:10094000009709F461C0EFE9FFE03197F1F700C0CB
:1009500000000197F5CFE22FF0E0EA56FE4F249019
:10096000822F86958695869590E0FC01EA57FE4F8A
:1009700064902770712C022E02C0759467940A94BB
:10098000E2F7F1E06F227724FC01EA58FE4F8490F1
:10099000912C022E02C0959487940A94E2F731E0DC
:1009A00083229924FC01EA59FE4FC490D12C02C045
:1009B000D594C7942A95E2F781E0C822DD2461141A
:1009C000710419F081EE0E9449238114910419F0F9
:1009D00086EE0E94492360E070E0822D0E9405248B
:1009E0008114910419F086EE0E94F82261147104BA
:1009F00019F081EE0E94F822C114D10429F060E0C0
:100A000070E08CE20E9405240F5F1F4F49CFF80170
:100A1000E851FC47E730F10508F05DC404C106E287
:100A200021EE41EE6AE17CE7C7010E9462188091E5
:100A30001002877009F470C4F7018581882309F4D6
:100A40006BC48091B60182FF67C482E00E944B12A2
:100A500063C4F801E851FC47E730F10508F4E3C04E
:100A60001092B602980130572332310508F003C1C5
:100A700084E090E00E94F2259093B6018093B50146
:100A8000F801E150F047E232F10520F4EA5AFF4F55
:100A90000C94D3268091B5018160ACC08091B601E1
:100AA0008860B4C08091B5018260A4C08091B50116
:100AB00020C08091B50188609DC08091B6011EC0A4
:100AC0008091B6018260A2C08091B501806192C020
:100AD0008091B50180628EC08091B50180648AC02A
:100AE0000E94D1228091B501806884C08091B501B7
:100AF000886084607FC08091B6018260816086C01A
:100B00008091B5018E7F76C08091B601877F7EC0CF
:100B10008091B5018D7F6EC08091B50120C080911C
:100B2000B501877F67C08091B6011EC08091B60174
:100B30008D7F6CC08091B5018F7E5CC08091B501C6
:100B40008F7D58C08091B5018F7B54C00E94D12207
:100B50008091B5018F774EC08091B501877F8B7FE3
:100B600049C08091B6018D7F8E7F50C08091B501C4
:100B700082FB222720F991E0922790FB82F990FBDB
:100B800083F938C08091B601982F909591708E7F2F
:100B9000892B90FB81F93AC08091B50186FB222711
:100BA00020F991E0922790FB86F924C00E94D1227F
:100BB0008091B50187FB222720F991E0922790FBD5
:100BC00087F918C061E001C060E08EE090E00E940B
:100BD00008261EC08091B50184FB222720F991E0F0
:100BE000922790FB84F906C08091B501982F9095CB
:100BF00090FB80F98093B5010BC08091B60183FB17
:100C0000222720F991E0922790FB83F98093B60187
:100C10006091B5017091B60184E090E00E942626B3
:100C20000E94D12204CFE858FF4F0C94D32607E24C
:100C300025EE45EE6BE17CE7F7CE06E221EE40EED5
:100C400068E17CE7F1CE07E225EE44EE69E17CE75E
:100C5000EBCE06E221EE42EE6CE17CE7E5CE07E268
:100C600025EE46EE6DE17CE7DFCE08E221E045EEC1
:100C70006EE17CE7D9CE80911B020631FCE71F07AD
:100C800009F41DC38272F801E052F847EB30F10518
:100C900008F05CC0E158FF4F0C94D32680917A0293
:100CA00080FF19C0282F2E7F20937A0230917B027B
:100CB00040917C0250917D0260917E0270917F0292
:100CC00080918002909181020E94861F1092DE0224
:100CD0000E94071FACCE816080937A0261E0869506
:100CE00086950E94B420A3CE882329F00E94042177
:100CF0009ECE8823D9F30E940F2199CE882329F014
:100D00000E94A02094CE8823D9F30E94AA208FCEDF
:100D1000882329F00E9486208ACE8823D9F30E9456
:100D2000932085CE882329F00E946C2080CE8823D2
:100D3000D9F30E9479207BCE882329F00E94AC1F32
:100D400076CE8823D9F30E94C61F71CE0737FCE701
:100D50001F0711F481E005C008372CE7120749F49A
:100D600082E00E949F2243E062E081E00E946314DF
:100D70005ECE9801205E324520323105A8F49111F3
:100D800015C00F7181E090E0FC0102C0EE0FFF1F63
:100D90000A95E2F78F016E2F83E090E00E9408260B
:100DA000802F0E94AB2243CE9923E9F10330FCE768
:100DB0001F0729F148F401153CE7130791F00130B2
:100DC0008CE7180711F12FC00B359CE7190741F18B
:100DD0000C35ECE71E07E1F00A351C4721F581E0F0
:100DE00020C00E94D1222FEF34E38CE0215030400C
:100DF0008040E1F700C000000E941E1718CE6FEF80
:100E00007FEF80E090E00E9426260E94E9240FCE2A
:100E10008091B60182FB882780F991E0892701C083
:100E200080E00E946212F701858100811181882390
:100E300049F0C8010E94EA21D82E682FC8010E94FB
:100E40005A2204C0C8010E942622D82EB8018D2D36
:100E50000E944E100E945C10D82E192FA82EF70168
:100E60000581C680C2949FE0C922809110028770DC
:100E700001F10023F1F0812F807F803469F080E25E
:100E80008D0D8830B0F0812F807E803229F4F1E022
:100E9000FD1578F4CC2069F08091B60182FF09C07D
:100EA00082E00E944B12809110028770BB24B394A1
:100EB0008111B12C912E92948FE09822892D90E08F
:100EC0008C30910508F0D1C1FC01E657FF4F0C941E
:100ED000D326812F807F1F70882311F01295107FF9
:100EE0000023B9F0112309F4AEC180E28D0D8830E2
:100EF00010F0A11006C090911B02192B10931B0239
:100F000005C090911202192B109312020E94111227
:100F10009AC18D2D0E94F822112309F4A6C180E206
:100F20008D0D883088F1AA2079F1109590911202E8
:100F30001923109312022BC0812F807F1F708032E3
:100F400011F01295107F8D2DAA2029F021E0A21614
:100F500009F44CC057C08091B60182FD1BC000232C
:100F600069F0112339F090911B02192B10931B0289
:100F70000E94111280E00E94492377C180E00E9404
:100F8000F822112309F471C1812F0E940A120E94D4
:100F900011126BC1002381F0CC20C1F131E0C312EA
:100FA00064C190911102812F8923181709F45DC142
:100FB000192B1093110259C1C11057C1812F0E94E2
:100FC000E72280911102912F982329F0912F90957B
:100FD0008923809311022091A901812F822309F492
:100FE00044C1109521232093A9013FC1002329F07A
:100FF00085E08C1508F439C109C094E09C1508F40B
:1010000034C115C0002331F0C1101DC1812F0E94D1
:10101000EE222BC1CC2059F0893309F023C1EFEF28
:10102000F7EE23E0E150F0402040E1F719C1812FB5
:101030000E94E7221AC1812F86958695837019F048
:10104000813061F012C1002321F08D2D912F93701A
:1010500002C080E090E00E94F3170FC1002321F04E
:101060008D2D912F937002C080E090E00E94CE17EA
:1010700004C1812F8370A9F50111FBC04D2D42954C
:1010800046954770440F440F8D2D8F7090E09C0162
:10109000042E01C0220F0A94EAF7D4FE08C08FE0A4
:1010A00090E001C0880F4A95EAF7809501C080E082
:1010B000169516951370123069F088F490911C0201
:1010C000113019F0822B892302C0922B892B0E94A8
:1010D000AB22CFC0822B90911C028927F8CF822BA4
:1010E000F6CF002319F0812F817001C086958823E7
:1010F00009F4BFC04D2D429546954770440F440FEB
:101100008D2D8F7090E09C01042E01C0220F0A9457
:10111000EAF7D4FE08C08FE090E001C0880F4A953E
:10112000EAF7809501C080E016951695137012308D
:1011300059F078F49091B401113019F0822B892381
:1011400009C0922B892B06C0822B9091B40189276C
:1011500001C0822B0E948F228CC01F70002339F0A7
:10116000812F0E949F228D2D0E94EE2282C08D2D04
:101170000E94E722812F0E9492227BC08D2D32EFA8
:10118000A31681F13A1538F090EFA91659F0E1EF66
:10119000AE1619F154C0F3EFAF1659F124EFA216B1
:1011A000C1F04DC0002381F034E03C1508F45DC06F
:1011B0001F7181E090E0012E01C0880F0A94EAF7C8
:1011C0009091B401892720C085E08C1508F44DC0AA
:1011D000EFCF8091B60182FD1AC0002329F0812F44
:1011E0008F7120C00023D9F3812F8F710E9492222A
:1011F0003CC0002341F01F7181E0012E01C0880F27
:101200000A94EAF701C080E00E948F222EC00023DA
:1012100061F0812F8F7198E0899F900111242360E4
:10122000209310020E949F2220C081E00E944B1256
:10123000E1E0EC15D0F482E00E944B1216C00023CE
:1012400021F0CC2061F28D2D96CECC2069F289332D
:1012500049F4FFEF27EE33E0F15020403040E1F752
:1012600000C000008D2D0E94F82288EF890D843087
:1012700020F40E9418180E941D24BB20A9F0809120
:10128000100280FD11C0F70115828695869586951E
:101290000E949F22C7010E94B5038091100286958B
:1012A000869586950E94922220E0F7014081518127
:1012B00062817381848195810E9434242DC08A7A51
:1012C00091E009F490E09093A801811112C089E2A5
:1012D0000E94B5170BC006312CE7120771F48091FC
:1012E000A801811108C089E20E94A9170E94111269
:1012F0009ECB85E3EDCF85E3F7CF07373CE71307B8
:1013000011F481E006C008378CE7180709F031CDE9
:1013100082E00E94922227CD2896E2E10C940B27CE
:10132000A6E2B0E0E6E9F9E00C94EF2685B7806824
:1013300085BF85B7806885BF84B7877F84BF0FB6B8
:10134000F894A89580916000886180936000109265
:1013500060000FBE90E080E80FB6F89480936100C3
:10136000909361000FBE81E08093120189E69EE0B8
:101370009093A7018093A6010E945C1D0E947B1D93
:101380008091E20084608093E20078948091CD02A5
:101390008823A1F01091E9001F709091EC00892F33
:1013A000817090FD80E8182B1092E9008091E80090
:1013B00083FD0E94401A1F701093E90082E084BDF3
:1013C00093E095BD9AEF97BD80936E000E944918F7
:1013D000811102C00E945E1900E211E0D8018D91D6
:1013E0008D018F3F11F00E94760FB1E005321B078F
:1013F000A9F705E211E082E3E82E81E0F82EF8017A
:1014000081918F018F3F11F00E94760FE016F10657
:10141000B1F78AE0E5ECF1E0DF01282F1D922A9573
:10142000E9F7EAEAF1E0DF011D928A95E9F780E049
:1014300090E00E94F225853E9E4F21F40E944918BB
:10144000811102C00E949D1182E090E00E94E4257B
:101450008093B30284E090E00E94F2259093B6015D
:101460008093B5010E948D0FEFEFF6E721E0E15088
:10147000F0402040E1F700C000000E948D0F8091F5
:10148000C50180FF08C06FEF7FEF80E090E00E9411
:1014900026260E941E1783E090E00E94E4250E9409
:1014A000AB22529A5A98519A5998509A58988091CA
:1014B000B70181117FC088E090E00E94EC254B01CC
:1014C0005C0183E290E00E94E425282F30E040E0B8
:1014D00050E060E070E080E090E000E20E942627AB
:1014E000282939294A295B2920937A0230937B02E3
:1014F00040937C0250937D0260937E0270937F0242
:1015000080938002909381022C7F09F041C025E0F6
:1015100020937A0210927B023FEF30937C0230934B
:101520007D0210927E0230E04FEF5FEF60E00E949C
:10153000861F88E090E00E94EC256B017C0183E22D
:1015400090E00E94E425282F30E040E050E060E089
:1015500070E080E090E00E942627B22FA32FF42FA6
:10156000E52F5B0197018601BC29A12BF22BE32B10
:10157000B0937A02A0937B02F0937C02E0937D0209
:1015800060937E02B0927F028093800290938102EA
:101590000E94721F1092DE020E94961480917A02BD
:1015A00080FF05C060E0869586950E94B42081E0AA
:1015B0008093B70184E091E09093BA028093B902DE
:1015C000B8E14B2E512C8E010F5F1F4F8091CD0241
:1015D000853009F060C08091CD02853009F04CC0A3
:1015E0008091CD02843009F439C080E00E941D242E
:1015F0001092DE028091B90181110EC081E08093CA
:10160000B90180917A02982F91709093B8018E7FE2
:1016100080937A020E94071F1092BD0290E40FB6D9
:10162000F894A895409260000FBE9093600083B735
:10163000817F846083BF83B7816083BF78948895FE
:1016400083B78E7F83BF0FB6F894A8958091600012
:10165000886180936000109260000FBE0E948D0F21
:10166000E5ECF1E081919191892B09F00CC3A1E0A7
:10167000EF3CFA07B9F7AFCF0E94D1220E941818A9
:101680000E941D241092B9018091B80181110E941D
:10169000F9200E94F01E0E948D0FFAEBEF2EF1E070
:1016A000FF2EA5EC6A2EA1E07A2ED301F70121913D
:1016B00031918D919D918227932721E0E43CF2079F
:1016C00019F0892BA1F305C0892B19F40E94791117
:1016D0003FC0312CD3018D909D903D01F701A0803A
:1016E000B180A824B924A114B10449F1212CCC243F
:1016F000C394D12CC5018C219D21892BB9F029A23D
:101700003AA20E9474179CA38BA3F1E0FDA391E081
:1017100094012C213D21232B09F490E09EA349A1A3
:101720005AA16BA17CA18DA10E9459242394CC0CB9
:10173000DD1C2DE02212DECFD7018D929C923394D6
:10174000B2E0EB0EF11CE5E03E12C4CF0E94681738
:101750008091DE02882309F4ABC08091DD02E09124
:101760007A02E695E695E81BE093D902823059F4B7
:10177000F0E0E95DFD4FE491EE2EF12C6EE5C62E12
:101780006FE1D62E70C0863059F4F0E0EC5DFD4F6D
:10179000E491EE2EF12C5EE4C52E5FE1D52E63C000
:1017A000893061F4E695F0E0EF5DFD4FE491EE2EB7
:1017B000F12C42ECC42E41E2D42E55C08F3061F49E
:1017C000E695F0E0E25EFD4FE491EE2EF12C37E677
:1017D000C32E31E2D32E47C0853159F4F0E0E55EE7
:1017E000FD4FE491EE2EF12C2BE1C22E21E2D22E00
:1017F0003AC08831F9F0833249F4E9E1F2E0E5904A
:10180000F49096EFC92E95E1D92E2DC08432D1F0F7
:10181000853209F58E2F63E00E949F26E92FF0E0C4
:10182000EA5EFD4FE491EE2EF12C8DEBC82E84E1A3
:10183000D82E19C0A8E2EA2EF12CBEE7CB2EB5E1D6
:10184000DB2E11C0E4EFEE2EFF24F394FFE4CF2E45
:10185000F5E1DF2E08C060EDE62E67E0F62E7FEEA4
:10186000C72E7EE1D72E8091DA02882361F0109294
:10187000DA020E9474179093D8028093D7021092D4
:10188000DC021092DB020E947417E091D702F09103
:10189000D8028E1B9F0B8F3F9F4750F4EE0EFF1E0A
:1018A000F092D802E092D70287ED92E0F601099516
:1018B0000E941818F82E8091C401F81639F0F092A1
:1018C000C4010E9468178F2D0E941D248091CD02B3
:1018D000843009F07BCE83E08093E9008091E800BA
:1018E00082FF74CE8091E80085FF23C00E94BC1E59
:1018F00081111DC050E2E52EF12CCE0101966C0144
:1019000009C08091F100D6018D936D01B1E0EB1A11
:10191000F10869F08091E80085FDF3CF8091E8003F
:101920008B778093E8000E94BC1E882399F391E096
:1019300001C090E08091E8008B778093E8009923C4
:1019400009F444CE2981822F90E0FC013197E331E4
:10195000F10508F08FC1EA56FF4F0C94D3261A8286
:101960008CE0F3C08A81823009F4AAC150F481303E
:1019700009F080C10E9468179B838C837D836E83EE
:101980007BC1833041F0843009F074C11B821C821A
:101990001D821E8271C16B81DE01119680E090E094
:1019A000262F30E0A901480F591F4530510508F096
:1019B00063C1E62FE80FF0E0EE0FFF1FEB53FE4F81
:1019C0004081518113965C93139714964C9314970E
:1019D000019612968E30910529F74EC18A81823088
:1019E00019F0853051F046C16B817C818D819E81DB
:1019F0000E94D9260E9425183FC180917A0280FF5B
:101A00000AC080917A028E7F80937A021092DE0261
:101A10000E94071F31C10E94F9202EC14C816B81A9
:101A20008A810E946E199D8352C12D813E81322789
:101A3000232732274C816B818A810E9402191CC1A5
:101A40000E94291919C18A81823009F013C12830F6
:101A5000B9F1293009F460C08B818230F9F098F433
:101A6000813009F009C18C81EFEF8E9FC0011124F4
:101A70006FEF70E00E94AB26462F20E060917C0261
:101A800080917B021AC08330A1F0843009F0F4C049
:101A900020E040917D026D818C810FC08C81882374
:101AA00009F4AFCF0E94F92060E08C810E94B4203D
:101AB000E3C08C8180937E02DFC00E94EF1FDCC0F8
:101AC0008B818230E1F078F4813009F0D5C08091CB
:101AD0007D02FFEF8F9FC00111246FEF70E00E9425
:101AE000AB266C83C9C0833099F0843009F0C4C040
:101AF00080917B028C8380917C028D83BDC080911C
:101B00007A0280FF03C08695869504C080E002C0FB
:101B100080917E028C83B0C020917A0230917B024A
:101B200040917C0250917D0260917E0270917F0213
:101B300080918002909181020E94861F9DC020E1C9
:101B40002A839AC082E08A8382E58B8395C0EA80EB
:101B5000FB80FE24EF24FE24CC80D12C5801C70149
:101B600082559E4F9501201B310B2C153D0508F029
:101B700083C0A2E5EA16A2E0FA0628F40E94E42552
:101B8000F501848303C0D50114961C92BFEFEB1AB4
:101B9000FB0AEFEFAE1ABE0AE2CFEA80FB80FE241A
:101BA000EF24FE24CC80D12C5801C70182559E4FD2
:101BB0009501201B310B2C153D0508F05DC0F2E5A9
:101BC000EF16F2E0FF0628F4D50114966C910E94FE
:101BD0000826BFEFEB1AFB0AEFEFAE1ABE0AE5CFFD
:101BE0000E94F21849C083E08A8346C0EA80FB80E5
:101BF000FE24EF24FE24CC80D12C5801C701889606
:101C00009501201B310B2C153D05B0F5F6E8EF16BC
:101C1000F1E0FF0630F40E94E425D50114968C9380
:101C200002C0F5011482FFEFEF1AFF0A2FEFA21A8C
:101C3000B20AE4CFEA80FB80FE24EF24FE24CC80AD
:101C4000D12C5801C70188969501201B310B2C150A
:101C50003D0590F4A6E8EA16A1E0FA0620F4F501A5
:101C600064810E940826FFEFEF1AFF0A2FEFA21AE5
:101C7000B20AE8CF8FEF898340E250E0B80182E0FA
:101C80000E94C516A3CC8091CC02882309F4A3CC72
:101C9000B0E1B9BDE2E1E9BD09B400FEFDCF80913C
:101CA000D8008F7D8093D8008091E000826080937F
:101CB000E0008091E00081FDFCCF0E94D1228BCC1E
:101CC00087E290E00E94E4251B821C821D828E83A5
:101CD000D3CF80E008959091B50192FF10C041E00C
:101CE000282F2471243009F040E031E0282F28719A
:101CF000283009F030E0431711F02CE0822793FFE1
:101D000010C041E0282F2471243109F040E031E077
:101D1000282F2871283109F030E0431711F02CE00A
:101D200082273091B60130FF10C051E0282F217179
:101D3000213009F050E041E0282F2871283009F0C7
:101D400040E0541711F029E0822731FF10C041E034
:101D5000282F2171213109F040E031E0282F28712E
:101D6000283109F030E0431711F029E0822794FD73
:101D7000877E08958238910569F1B0F48133910529
:101D800009F475C048F48932910509F467C08A32B4
:101D9000910509F471C008958533910509F459C07E
:101DA00089339105B9F00895833E910589F138F49E
:101DB000803E9105D1F0823E910529F10895863E3D
:101DC0009105C9F1873E9105D9F1843E910509F04D
:101DD0006CC027C02091B50120FD57C021FD55C022
:101DE0002091B60123FD5BC008958091B50180FD6F
:101DF00048C08091B60180FF48C08091B50184FD44
:101E000046C083EE51C08091B50182FF3CC0F5CF42
:101E10008091B50182FD37C08091B60180FD35C04B
:101E2000ECCF8091B60181FF36C08091B50184FD71
:101E30002EC087EE39C08091B50183FF2AC0F5CF4F
:101E40008091B50183FD25C08091B60181FD23C03D
:101E5000ECCF8091B50185FD22C01FC08091B501F6
:101E600085FD1BC08091B60183FF19C00AC0809117
:101E7000B50186FD16C017C08091B50186FD13C05F
:101E800010C089E311C082EE0FC080EE0DC080E06B
:101E90000BC086EE09C084EE07C085E305C089E269
:101EA00003C08AE201C081E390E0089520910F020F
:101EB0009091D60157E02917A9F030E0529FF00128
:101EC000539FF00D1124E952FE4F7181761306C025
:101ED0007081781303C07581741306C02F5F3F4F64
:101EE0002770E9CF80E0089581E00895F894E82F05
:101EF000E295EF70F0E031A1282F2F7081E090E0A3
:101F000001C0880F2A95EAF7982F9095932391A303
:101F100092A1892B82A378940895AAE0B0E0E3E926
:101F2000FFE00C94F126AE014F5F5F4F7A018AE02B
:101F3000FA0111928A95E9F700E211E06A0195E24F
:101F4000492E91E0592E66246394712C32E3832E3E
:101F500031E0932EF80180818F3F09F446C0F89458
:101F6000E82FE295EF70F0E021A18F70A30102C08D
:101F7000440F551F8A95E2F7CA01922F982B91A31F
:101F800092A18095892382A3789400C0E5E2F1E0D4
:101F900021E030E0A12CB12C41914F3F89F0A42FDA
:101FA000A295AF70B0E090968C9190E04F7002C017
:101FB000959587954A95E2F780FD02C0C90102C058
:101FC00080E090E0A82AB92A220F331F8E169F06C0
:101FD00019F7F80180818F3F11F00E94760FF0EA27
:101FE000FA95F1F7F601B182A0820F5F1F4FF2E080
:101FF000CF0ED11C4016510609F0ACCF4AE050E09C
:10200000B7018AEA91E00E946A27892B91F08AE061
:10201000F701AAEAB1E001900D928A95E1F781E01B
:10202000809321020E9474179093200280931F02D4
:1020300017C080912102882399F020911F023091CE
:1020400020024FB7F8948091BE029091BF02A091F8
:10205000C002B091C1024FBF821B930B059710F4D1
:1020600080E018C04AE050E06AEA71E085EC91E057
:102070000E946A27892B59F08AE0EAEAF1E0A5EC90
:10208000B1E001900D928A95E1F781E001C080E016
:10209000109221022A96E0E10C940D27753048F445
:1020A0006D3038F4833028F4462F672F0E946E1964
:1020B000089580E090E008951F93CF93DF930E94EE
:1020C000BA0EEC01C11580E5D807E8F5C11590E41A
:1020D000D90708F0A8C0C03ED10530F5CD3CD105E8
:1020E00008F094C0C83AD10578F4C53AD10508F093
:1020F00083C0C130D10509F47CC008F4F2C0C430FB
:10210000D10508F0F1C0EDC0C33CD10508F0E9C02D
:10211000C85AD0E0CC0FDD1FCB5CDE4F0990D881D0
:10212000C02DCE019464E1C0C11580E2D80708F04B
:10213000CBC0C11591E0D90708F06BC0C83ED105EE
:1021400008F4D2C0CEC0C03682E5D80728F5C03426
:1021500092E5D90708F079C0C03282E5D80708F0C7
:102160006CC0C11592E5D90708F481C04C2F469583
:10217000469580E2489FA0011124C37021E030E021
:10218000C90102C0880F991FCA95E2F7EA01C82B5E
:10219000D92BCE019D68A9C0C03A82E5D807B8F412
:1021A0008C2F8F71C03892E5D90708F07BC08695D7
:1021B000869590E2899F90011124C37081E090E0A0
:1021C00002C0880F991FCA95E2F79A6868C0C03CA0
:1021D00082E5D80708F46DC0C03E92E5D90708F043
:1021E00080C0CF71DD27DC2FCC27CE01806F906AB5
:1021F0007CC081E090E079C0C55AD0E0CE5CDE4F73
:102200008881C82FD0E0CE0190646FC0CE01906568
:102210006CC08D2F0E946B0E182FCE0199270E9443
:10222000BA0E1F715CC0CE0199270E94BA0ECC274E
:10223000DF70D06A8C2B9D2B58C0CF71D0E0DC2F83
:10224000CC27CE01816F906A50C08C2F8F718695FC
:10225000869590E2899F90011124C37081E090E0FF
:1022600002C0880F991FCA95E2F79C6818C08C2F8E
:102270008F710E946B0E95E0D695C7959A95E1F700
:10228000CF70D0E0DC2FCC27282F30E084FF05C0B2
:1022900084E0220F331F8A95E1F7D069CE01822BAB
:1022A000932B23C090E0D82FCC27CE01846F906A67
:1022B0001CC08C2F8F710E946B0E8F7190E0D82FF5
:1022C000CC27CE01906211C08D2F8F710E946B0EB2
:1022D000182FCE0199270E94BA0E1F719062912B80
:1022E00004C080E090E001C0CE01DF91CF911F914A
:1022F0000895A6E0B0E0EFE7F1E10C94FD260E941E
:1023000074178C0180911D0290911E020817190705
:1023100081F019821A820E947417682F49815A81AC
:10232000792F80E090E00E94592410931E020093C0
:102330001D022696E4E00C941927A8E0B0E0E3EA39
:10234000F1E10C94FF2665EE7EEF80E090E00E94C4
:10235000262660E082E090E00E94082681E08093DB
:102360001C0261E083E090E00E94082660E074E1D6
:1023700084E090E00E94262660E086E090E00E94E3
:10238000082660E087E090E00E94082640E050E0E8
:10239000BA0188E090E00E941A2660E083E290E0B3
:1023A0000E94082660E08CE090E00E94082660E031
:1023B0008DE090E00E94082619821A821B821C82FE
:1023C0001D821E821F82188648E050E067E170E09F
:1023D000CE0101960E94F82540E050E0BA018FE15D
:1023E00090E00E941A2680E00E942A180E945E193E
:1023F00040E050E0BA018FE090E00E941A2640E0F1
:1024000050E0BA0183E190E00E941A262896E2E0AB
:102410000C941B27809590911B02892380931B02AB
:10242000089590911B0280911202892B90911102C4
:10243000992379F0892BE4E2F2E027E090E0215043
:1024400029F031913323D9F39F5FF9CF9111109285
:1024500011028093220248E050E063E172E082E2E0
:1024600092E00E946A27892BA9F088E0E2E2F2E07C
:10247000A3E1B2E001900D928A95E1F7E091B902F3
:10248000F091BA02309731F00280F381E02D82E2C0
:1024900092E0099508959091100280958923809388
:1024A0001002282F277069F4981759F09091B601FF
:1024B00092FF07C08695869586950E94922210927B
:1024C000100208959091B60192FB222720F9281757
:1024D00079F080FB92F99093B6016091B50170910B
:1024E000B60184E090E00E94262682E00E944B1212
:1024F000089580910F029091D601891719F08F5F8E
:102500008770FBCF0895CF93DF938091D50182959B
:102510008F7009F04EC08091D401882309F449C01E
:1025200080910F024091D6015091D0016091CF016E
:10253000C091D101D091D20177E08417D1F190E020
:10254000789FF001799FF00D1124DF01A952BE4F51
:1025500014962C911497222349F111962C911197DE
:10256000251324C02C91261321C015962C91159764
:1025700021111CC012962D913C9113972C1B3D0BE1
:10258000283C310598F48091D5018F70806180934B
:10259000D501E352FE4F80818F70806180838FEC84
:1025A00091E00E94B5030E94791203C001968770E2
:1025B000C4CFDF91CF910895A4E1B0E0E2EEF2E163
:1025C0000C94F5268C0186E0F801DE011F9601903F
:1025D0000D928A95E1F7F8018481E5809FEC892EC0
:1025E00091E0992E9091D301911120C0882309F494
:1025F00063C1EE2009F442C0C8010E94AE22F82E49
:102600008823E1F187E0F801D40101900D928A95C9
:10261000E1F78091D301813031F48091CF01909125
:10262000D0010E9419220E94831248C1F801D08073
:10263000C180A280B380F090D4012091D10130916B
:10264000D201FF2009F4E7C0A501421B530B483C0F
:10265000510508F09DC0882309F430C18091D5014F
:10266000282F207F9091D001222361F09C1509F43E
:1026700060C0C8010E94AE22811163C0C8010E94DF
:10268000B5031AC19C1113C09091CF019D110FC0C9
:10269000E1100DC08F7080618093D5018FEC91E0C7
:1026A0000E94B5038091D501F801868303C1E11032
:1026B0003AC040E06C2D8D2D0E94560F40E06C2DED
:1026C0008D2D0E94560FE82E8111F4C0DF86C88A36
:1026D0008F8598890E941922292F22952F702430E6
:1026E00020F49F70223028F009C02A50223080F058
:1026F00014C0992349F0811107C013C0992321F018
:10270000F8019681907F69F0805E883030F409C0CE
:10271000803F38F0815F833020F0C8010E94B5030C
:10272000EF2CFE2CCBC08091D50181608093D50128
:10273000C1C09091CF019D119CCFE1109ACFF801BB
:1027400098C0EE2009F49ACF2091D501822F82956E
:102750008F7090E002978CF08091CF019091D00122
:1027600099878887BB86AA868091D3018C871D862E
:102770002E87CE0108960E94B50387E0F801AFECE2
:10278000B1E001900D928A95E1F70E94831294C006
:102790009091D501292F207F51F48FEC91E00E9478
:1027A000B50387E0F40111928A95E9F783C0882385
:1027B00009F484C08091D0018C110CC08091CF01AC
:1027C0008D1108C0E11006C0F8019683C8010E946F
:1027D000B5036AC0C8010E94AE22882309F44ECF17
:1027E000EE2009F44BCF2091D501822F82958F7076
:1027F00090E0029714F28091CF019091D0019A83DA
:102800008983BC82AB828091D3018D831E822F830A
:10281000CE010196B0CFA21AB30AF8ECAF16B104FC
:1028200008F042C0882309F447C0FE2CEE2009F4CA
:1028300025CF8091D0018C1129C08091CF018D11BD
:1028400025C09091D50190FD18C0892F82958F7079
:10285000282F30E02115310581F0F80196832F30C3
:10286000310541F08F5F982F9295907F86818F7010
:10287000892B8683C8010E94B50387E0F801AFEC7D
:10288000B1E001900D928A95E1F718C0C8010E944D
:10289000AE22811172CF8091D50181608093D501E4
:1028A000C8010E94B5030AC087E0F40111928A951D
:1028B000E9F704C0F12C02C0FF24F3948F2D649635
:1028C000ECE00C9411279091B40121E030E0F90183
:1028D00001C0EE0F8A95EAF7D90102C0AA0FBB1F0B
:1028E0006A95E2F7BD016E2B01C0220F4A95EAF707
:1028F000892F8623681303C0892F822B03C020955C
:10290000822F89230E948F2208950895089580912F
:1029100010010895FC01EE0FFF1F8E0F9F1FFC0199
:10292000EE57FD4F6183408322830895579A08959F
:102930008BB18F779BB190682FB7F894E2E8F2E003
:1029400032E0E23BF30789F0319148E09BB90000A7
:1029500000C037FF8BB9330F000000C000C000C0BB
:102960008BB900C04A9591F7EBCF2FBF8FE594E06C
:102970000197F1F700C000000895A0E0B0E0E3EC9B
:10298000F4E10C94F426FC018280748081E084835D
:10299000EBE2F2E09490EAEAF2E0E49100917D0249
:1029A0000695015810E0000F111F012F1127CAE2F0
:1029B000D2E0C12CD12CAA24AA94B12CE919EE2E74
:1029C000F12C22E0281530F080917B0288838091E1
:1029D0007C028983711003C01B821A824AC08B81DA
:1029E0008823F9F081508B832FEF829FC00111243F
:1029F0006C8170E00E94AB26FB01FF27E55DFD4F77
:102A00008491E82FE9192FEFE29FC0011124B7014B
:102A10000E94AB2680917D02689FB00111247A83C9
:102A200028C00E94D425B5010E94BF2680179107B7
:102A300004F582E0881588F40E94D425B5010E942F
:102A4000BF2688830E94D42520917C022695622F80
:102A500070E00E94BF26280F29831A8280917D0290
:102A6000843120F0893C18F088EC01C084E18C832B
:102A70008B8396014A81698188810E94E01F2FEF34
:102A8000C21AD20A259680E1C816D10409F099CF5E
:102A90000E94071FCDB7DEB7EDE00C9410270F930F
:102AA0001F93CF93DF938C01C0E0D0E0F8018481C5
:102AB000C830D1051CF4882339F002C0811104C04C
:102AC0009E0140917D0202C09E0140E060917C0227
:102AD00080917B020E94E01F2196C031D10531F721
:102AE0000E94071FF801848190E001968170992768
:102AF0008483DF91CF911F910F910895A0E0B0E002
:102B0000E4E8F5E10C94F526EC014C81042F10E08B
:102B10009801D8010E9490269B01AC010E945B267F
:102B20006B017C01E0E2F0E0E01BF10BA5E5B0E019
:102B30009B01AC010E945B264B015C019F01DF0100
:102B40000E94E0269B01AC010E9466269B01AC011D
:102B50002C0D3D1D4E1D5F1DC501B4010E946E264A
:102B6000822F022F2A3228F493E0299F900111240A
:102B70000DC025E530E0281B3109C901880F991FD8
:102B8000280F391F37FF02C02F5F3F4F359527951C
:102B9000122F1095E12CF12C85E5D82ED01AE1FCEE
:102BA00002C08D2D01C0802F9701412F60917C02C2
:102BB0000E94E01F8FEFE81AF80A90E1E916F1048D
:102BC00071F70E94071F8C81811102C091E003C040
:102BD000803219F49FEF90930E0190910E01890FAE
:102BE0008C83CDB7DEB7ECE00C941127CF93DF9345
:102BF000EC0140917D029C8190FF02C0842F01C0B6
:102C000080E091FF02C0642F01C060E092FF40E0CD
:102C10000E941F1F8C8190E00196877099278C83FA
:102C2000DF91CF9108958091CF0287FF11C08091ED
:102C3000E80082FD05C08091CD028111F8CF11C05E
:102C40008091E8008B770BC08091CD02882349F0FA
:102C50008091E80080FFF8CF8091E8008E77809324
:102C6000E8000895982F973068F59093E900981739
:102C700039F07091EC002091ED005091F00003C00C
:102C8000242F762F50E021FD02C09F5FECCF3091C2
:102C9000EB003E7F3093EB003091ED003D7F3093B1
:102CA000ED003091EB0031603093EB007093EC005D
:102CB0002093ED005093F0002091EE0027FDE5CF2A
:102CC00080E008958F708093E90081E0089520915D
:102CD000D5023091D6022617370748F061157105E5
:102CE00039F42091E8002E772093E80001C0B90163
:102CF000FC0120E06115710579F18091CD028823F6
:102D0000F1F18530F1F18091E80083FD3CC08091C4
:102D1000E80082FD2EC08091E80080FFEBCF20917B
:102D2000F3008091F20090E0922B6115710551F053
:102D30008830910538F421912093F1006150710998
:102D40000196F3CF21E0089709F020E08091E80098
:102D50008E778093E800CECF2111CFCF0AC080912B
:102D6000CD02882361F0853061F08091E80083FD19
:102D70000AC08091E80082FFF2CF80E0089582E0EF
:102D8000089583E0089581E008950F931F93CF93F2
:102D9000DF938B01EA019091CD02943079F58F7029
:102DA0008093E9008FEF9091E800815095FD06C077
:102DB00095ED9A95F1F700008111F5CF8091E8002B
:102DC00085FF1CC00E94BC1E882361F08091E80032
:102DD0008E778093E80012C0F80181918F01809373
:102DE000F1002197209791F38091E80085FDF4CFC1
:102DF0008091E8008E778093E800E4CFDF91CF9157
:102E00001F910F91089543E050E0BC0184E00E94BF
:102E1000C5160895CF93DF93EC0148E050E0BC0164
:102E200081E00E94C51688E0FE01A3ECB2E00190AB
:102E30000D928A95E1F7DF91CF91089581E080931B
:102E4000E00080E28093D8001092C9008FE19EE4F8
:102E50000197F1F700C0000087E090EBDC01809360
:102E6000FC029093FD02A093FE02B093FF029CE04F
:102E700088E10FB6F894A895809360000FBE9093F8
:102E80006000FFCF78941F920F920FB60F9211241B
:102E90008F939F93AF93BF938091BE029091BF0297
:102EA000A091C002B091C1020196A11DB11D8093F5
:102EB000BE029093BF02A093C002B093C102BF9123
:102EC000AF919F918F910F900FBE0F901F9018950B
:102ED0002FB7F8946091BE027091BF028091C0023A
:102EE0009091C1022FBF08952FB7F8948091BE0230
:102EF0009091BF02A091C002B091C1022FBF08956E
:102F00001F920F920FB60F9211248F939F93AF933E
:102F1000BF938091BD02811113C08091BE02909138
:102F2000BF02A091C002B091C1024196A11DB11D86
:102F30008093BE029093BF02A093C002B093C102DF
:102F4000BF91AF919F918F910F900FBE0F901F90E7
:102F50001895E2E2F2E09281891301C01282319663
:102F600092E0E832F907B9F70895A4E2B2E0EFEF92
:102F700090E02D91821789F0EF3F19F4211101C0E3
:102F8000E92F9F5F9630A9F7EF3F39F00E2E000C26
:102F9000FF0BEE5DFD4F828308950895A3E0B0E03E
:102FA000E4EDF7E10C94FF262091BB023091BC02C6
:102FB00028173907A1F09093BC028093BB02E091DF
:102FC000B902F091BA02309751F024E029839B8333
:102FD0008A830084F185E02DCE0101960995239620
:102FE000E2E00C941B27A3E0B0E0E9EFF7E10C94DA
:102FF000FF262091B7023091B80228173907A1F0B7
:103000009093B8028093B702E091B902F091BA02AE
:10301000309751F023E029839B838A830084F185D4
:10302000E02DCE01019609952396E2E00C941B2732
:10303000E091B902F091BA02309729F00190F08145
:10304000E02D0995089580E0089587E290E00E94C0
:1030500008260895CF93C82F811102C06FEF01C0D9
:1030600065E284E290E00E940826C11102C06FEF81
:1030700001C061E085E290E00E940826C11102C013
:103080006FEF01C064E186E290E00E940826CF91D4
:10309000089584E290E00E94E425853281F485E27F
:1030A00090E00E94E425813051F486E290E00E9495
:1030B000E42591E0843109F090E0892F01C080E09F
:1030C000817008950F931F93CF93DF93C42F122F16
:1030D000FC0185818823B1F04093B6020E947417E9
:1030E0009093B5028093B40280E28C0F883008F090
:1030F00074C0C77081E001C0880FCA95EAF70E94CA
:10310000EE226BC08091B602481349C02091B402F0
:103110003091B5024FB7F8948091BE029091BF02F2
:10312000A091C002B091C1024FBF821B930B883C9B
:103130009105A8F5D0E2D10FC117E9F080E28C0F1C
:10314000883040F4C77081E001C0880FCA95EAF763
:103150000E94E722D83080F581E0912F977001C05E
:10316000880F9A95EAF70E94EE22093359F560E537
:1031700070E089E32AC0093319F460E570E002C009
:1031800060E070E0802F0E940524D83030F5212FB8
:10319000277081E001C0880F2A95EAF70AC080E213
:1031A0008C0F8830D0F4C77081E001C0880FCA95B9
:1031B000EAF70E94E72211C0093351F460E570E09C
:1031C00089E309C060E070E0802F0E940524DFCF12
:1031D00060E070E0802F0E940524DF91CF911F9165
:1031E0000F910895CF93DF93CEEAD1E060E0CE0156
:1031F0000E9408262196C11584E0D807B9F7DF910F
:10320000CF9108951F93CF93DF93962F8330E8F4E7
:103210006530D8F44D30C8F4632F122FC42FD0E09E
:10322000CC0FDD1F2AE1929FC00DD11D112492E821
:10323000899FC00DD11D1124CE0188960E940826B9
:10324000612FCE0189960E940826DF91CF911F91B0
:103250000895A0E0B0E0EFE2F9E10C94F726A12C8C
:10326000E12CF12CB12C00E010E0C0E0D0E06701CF
:10327000C00ED11EFE01EE0FFF1FEC0DFD1DE55D22
:10328000FC4F259134914C2F6B2D8A2D0E940219F1
:103290002196CD30D10571F7065E1F4FB39485E0BE
:1032A000B812E3CF82E8E80EF11CA39483E0A812E1
:1032B000D9CFCDB7DEB7EAE00C94132780E00E94A7
:1032C0002A1860E070E0CB010E9425180E9429199D
:1032D0000E94F21881E00E942A1808950F931F930C
:1032E000CF93DF93833008F56530F8F44D30E8F480
:1032F000C42FD0E0CC0FDD1F2AE1629FC00DD11D8D
:10330000112432E8839FC00DD11D1124CE0188966F
:103310000E94E42590E0182F0027CE0189960E9494
:10332000E4259801282BC90102C080E090E0DF91DC
:10333000CF911F910F9108958B3109F473C058F507
:103340008B3009F497C078F4863009F446C020F435
:10335000853009F44CC092C0873009F455C08830DC
:1033600009F488C08BC0803109F46FC068F48E30D6
:1033700009F084C08091B30282FB222720F991E0FA
:10338000922790FB82F957C0863109F473C08931C6
:1033900009F470C073C08A32E9F060F4873209F42E
:1033A0006BC028F48E3108F469C08D5159C0893240
:1033B000F1F064C0833450F48A3308F050C0853390
:1033C00009F45AC0883309F455C058C0833409F44D
:1033D00053C054C00E949D114DC08091B302817FA3
:1033E0008E7F8093B30281E08093B20208950E94A1
:1033F000D1222FEF84E39CE0215080409040E1F700
:1034000000C000000E941E178091B302982F909573
:10341000917090FB80F98093B30291112BC0897F4A
:10342000877F10C08091B30281FB222720F991E0B1
:10343000922790FB81F98093B3029923D9F0809170
:10344000B30281608093B30215C08091B30283FB05
:10345000222720F991E0922790FB83F9ECCF895342
:1034600091E001C0990F8A95EAF7892F0E94AB225B
:103470000E94D12281E0089581E0F8CF80E0089594
:10348000AAE2B0E0E6E4FAE10C94FE26EFECF2E00A
:1034900087ED92E02091F10021938E179F07D1F7DD
:1034A0008091D002833009F463C030F4813071F030
:1034B000823009F4A2C0B9C08A3009F48EC08B30C2
:1034C00009F46EC0893009F0B0C020C08091CF02ED
:1034D000813A09F0AAC08091E800877F8093E800D4
:1034E0008091D3029091D402892B21F468E083EC7F
:1034F00092E003C060E080E090E070E00E94671618
:103500008091E8008B778093E8008FC08091CF0294
:10351000813209F08AC08091D3029091D402009741
:1035200019F0029709F081C08091E800877F8093AD
:10353000E8008091E80082FD05C08091CD028111F4
:10354000F8CF73C02091F3008091F20090E0922BAD
:10355000029731F48091F100813011F0863021F42E
:103560008091F100809310018091E8008B7759C021
:103570008091CF02813A09F058C08091D302909196
:10358000D402892B09F051C08091E800877F809395
:10359000E8008091E80080FFFCCF809111013CC0E1
:1035A0008091CF02813209F040C08091D302909186
:1035B000D402892BD1F58091E800877F8093E800C1
:1035C0000E94131681E09091D102911101C080E018
:1035D000809311010E94D12228C08091CF028132B4
:1035E00021F58091E800877F8093E8000E94131600
:1035F0008091D20280930F0118C08091CF02813A4E
:10360000A1F48091E800877F8093E8008091E80032
:1036100080FFFCCF80910F018093F1008091E80042
:103620008E778093E8000E9413168091E80083FF54
:10363000E7C18091CF029091D002492F50E04A30EB
:10364000510508F0DDC1FA01E755FF4F0C94D32670
:10365000803821F0823809F0D3C108C08091CB02B4
:103660009091CC02992389F082600FC08091D3029F
:103670008F70873008F0C4C18093E9008091EB001F
:1036800085FB882780F91092E9009091E800977FE8
:103690009093E8008093F1001092F10071C1282FFF
:1036A0002D7F09F0ADC1882319F0823061F0A8C1E7
:1036B0008091D102813009F0A3C1933009F080E0FC
:1036C0008093CC022EC08091D10281112AC08091BA
:1036D000D3028F702FEF280F263008F091C180930E
:1036E000E9002091EB0020FF1CC0933021F4809171
:1036F000EB00806214C09091EB0090619093EB001E
:1037000021E030E0A90102C0440F551F8A95E2F77D
:103710004093EA001092EA008091EB008860809369
:10372000EB001092E9008091E800877F8093E80029
:103730000E94131665C1811163C11091D1021F77D8
:103740008091E3008078812B8093E3008091E800F2
:10375000877F8093E8000E9413168091E80080FF25
:10376000FCCF8091E30080688093E300111102C0D8
:1037700082E001C083E08093CD0242C18058823054
:1037800008F03EC12091D1023091D2022C3D53E08D
:10379000350779F583E08A838AE289834FB7F89405
:1037A000DE01139620E03EE051E2E32FF0E050937B
:1037B0005700E49120FF03C0E295EF703F5FEF7088
:1037C0008E2F90E0EA3010F0C79601C0C0968D931E
:1037D0009D932F5F243149F74FBF8091E800877F89
:1037E0008093E8006AE270E0CE0101960E946716BD
:1037F000B5C08091D3029091D402432F5527433016
:103800005105A9F068F44130510509F408C142306E
:10381000510509F0F5C08BE590E0E9E4F5E04BC017
:103820004132510529F14232510589F1E9C0C901FE
:10383000992781309105A1F058F0029709F0E0C076
:10384000E6EBF5E0E4918E2F90E0E6EBF5E030C09A
:10385000ECEEF5E0E4918E2F90E0ECEEF5E028C080
:10386000EAECF5E0E4918E2F90E0EAECF5E020C080
:103870008330910508F0C4C0880F991FFC01EC58F3
:10388000FE4F0190F081E02D89E090E014C083307C
:10389000910508F0B5C0FC01EE0FFF1FE259FE4F85
:1038A0000190F081E02DDC01A559BE4F8C9190E094
:1038B000009709F4A5C02091E800277F2093E80035
:1038C0002091D5023091D6028217930708F49C010B
:1038D00040E02115310589F18091CD02882309F45A
:1038E0003DC08530D9F18091E80083FD37C08091DB
:1038F000E80082FD2FC08091E80080FFEACF409170
:10390000F3008091F20090E0942B2115310559F0DD
:103910008830910540F444914093F1003196215054
:1039200031090196F2CF41E0089709F040E080911B
:10393000E8008E778093E800CCCF4111CDCF0AC04C
:103940008091CD02882351F0853041F08091E800CC
:1039500083FD04C08091E80082FFF2CF8091E800EF
:103960008B778093E8004CC0803809F049C0809183
:10397000E800877F8093E8008091CE028093F10079
:103980008091E8008E77D2CE81113AC08091D10229
:103990009091D202992702979CF58091E800877F49
:1039A0008093E8001091D1021093CE020E9413166A
:1039B000111106C08091E30087FD02C081E001C0C3
:1039C00084E08093CD0242E061EC81E00E943216F7
:1039D00042E261EC84E00E94321642E261EC82E055
:1039E0000E94321642E260EC83E00E94321680911F
:1039F000CD02843011F081E001C082E08093120199
:103A00008091E80083FF10C08091E800877F809359
:103A1000E8008091EB0080628093EB0005C082E1BA
:103A200090E0E4EAF5E047CFAA96E3E00C941A2789
:103A30001F920F920FB60F9211242F933F934F9323
:103A40005F936F937F938F939F93AF93BF93CF9326
:103A5000DF93EF93FF93C091E900CF708091EC006A
:103A6000D82FD17080FDD0E81092E9008091F0004D
:103A7000877F8093F00078940E94401A1092E900AA
:103A80008091F00088608093F000CD2BCF70C093C0
:103A9000E900FF91EF91DF91CF91BF91AF919F919D
:103AA0008F917F916F915F914F913F912F910F90E7
:103AB0000FBE0F901F901895E8EDF0E080818E7F8B
:103AC00080831092E2001092DA001092E100A0EEE2
:103AD000B0E08C9181608C9380818F77808319BC5A
:103AE000A7EDB0E08C918E7F8C9380818F7E808358
:103AF0001092C2020895A0E0B0E0E1E8FDE10C946C
:103B0000F926C8EDD0E088818F7E8883E7EDF0E06C
:103B100080818160808384E082BF81E08093C202E3
:103B200088818E7F888302EE10E0F8011082109267
:103B3000DA0081EEC82ED12CF601108288818F77B1
:103B4000888388818068888388818F7D888319BC79
:103B50001092CD021092CE021092CC021092CB02A3
:103B600090EEE92EF12CF70180818B7F8083888194
:103B70008160888342E060E080E00E943216F601B6
:103B800080818E7F8083F801808181608083808145
:103B900088608083F70180818E7F80838881806147
:103BA0008883CDB7DEB7E8E00C9415271F920F92FB
:103BB0000FB60F9211242F933F934F935F936F9300
:103BC0007F938F939F93AF93BF93EF93FF938091D6
:103BD000E10082FF09C08091E20082FF05C0809170
:103BE000E1008B7F8093E1008091DA0080FF2AC0A2
:103BF0008091D80080FF26C08091DA008E7F80936C
:103C0000DA008091D90080FF18C080E189BD82E18F
:103C100089BD09B400FEFDCF81E08093CD02809183
:103C2000C20281110FC00E945C1D0E947B1D809109
:103C3000E20084608093E20005C019BC1092CD02BE
:103C40001092C2028091E10080FF1AC08091E200D0
:103C500080FF16C08091E2008E7F8093E200809109
:103C6000E20080618093E2008091D80080628093BE
:103C7000D80019BC85E08093CD0283E080931201C7
:103C80008091E10084FF37C08091E20084FF33C05F
:103C900080E189BD82E189BD09B400FEFDCF80913C
:103CA000D8008F7D8093D8008091E1008F7E809333
:103CB000E1008091E2008F7E8093E2008091E2003B
:103CC00081608093E2008091CE02882311F084E02D
:103CD00007C08091E30087FD02C081E001C083E05E
:103CE0008093CD028091CD02843011F081E001C03B
:103CF00082E0809312018091E10083FF2CC08091CB
:103D0000E20083FF28C08091E100877F8093E1007B
:103D100082E08093CD021092CE028091E1008E7FEE
:103D20008093E1008091E2008E7F8093E200809199
:103D3000E20080618093E20042E060E080E00E9467
:103D400032168091F00088608093F00081E08093CB
:103D5000120180931101FF91EF91BF91AF919F915B
:103D60008F917F916F915F914F913F912F910F9024
:103D70000FBE0F901F9018952091E4003091E50040
:103D800095E64091EC00842F817040FF23C0809124
:103D9000E80080FD1DC08091CD02882399F0853018
:103DA00099F08091EB0085FD11C04091E4005091A5
:103DB000E5002417350729F3915011F09A01E1CF5E
:103DC00084E0089582E0089583E0089581E00895F5
:103DD00080E008954091E80042FFDDCF0895089506
:103DE00060917A026695669570E04BE050E083E161
:103DF00091E00E945D27892B19F481E08093DE0217
:103E00000E9474179093D8028093D7020895CF939D
:103E1000DF9380917A0280FF05C00E949814DF91A1
:103E2000CF910895C0E0D0E020E040E060E0CE0116
:103E30000E948A142196C031D105B1F7EECFFF92CE
:103E40000F931F93CF93DF9390917A0290FF11C04D
:103E5000F42E062F182FC0E0D0E02F2D402F612F19
:103E6000CE010E948A142196C031D105B1F70E947B
:103E7000071FCDB7DEB7E5E00C94182790917A02C2
